:0300000002039167
:0800030020312DC0D0024003A2
:08000B00C0D0202E1002400BB2
:0800130020122BC0D0024013A3
:08001B00C0D0020047026CFE98
:08002300C0D0201F1C02402385
:05002B00C0D002402BD3
:10003000026D3E202608C29630B2FDD296320220D2
:1000400040D21632022050201A0302401B022088A0
:100050006AC0160F126D1263696E065B06450628AC
:1000600017F517531585146A187E143F192B1915A7
:10007000191F17E61820182E18331827181A180DEC
:1000800017CE17A517D71929152D15AD15321691AD
:1000900017F6174D15C216D1183A18001910186323
:1000A000193F14331445126913B8144E19511955D8
:1000B0001959195F1965196B196F19731977197D1A
:1000C000199C11C213C766AA689D13190F8A1142A1
:1000D000114E07F6088A0A77010F0E0A080A08036C
:1000E00005040C0606060606060F0F0F0F0F0F0F6E
:1000F0000F0F0F0F0F0F0F53544F50225452592010
:10010000414741494E22524541445922202D204920
:100110004E204C494E452022088A12C00C9205D62A
:100120006C33698D6AAC6AB8048369750A830611F9
:100130000BB10BF813F50E1F6D2B6D310BBA0E239F
:1001400010A20F86057614196D140E2108771093EE
:10015000188E0C9A117F0DB411750D3718840EFB93
:1001600010230DCD11650C9C0BC60CD90B690C86A8
:100170000C8B6AC06C50127512796A8D0829804CFC
:10018000455481434C454152825055534883474F13
:10019000544F8450574D855048302E8655498755C9
:1001A0004F88504F50895052494E5489502E893FA4
:1001B0008A43414C4C8B44494D8C535452494E47D1
:1001C0008D424155448E434C4F434B8F5048312E06
:1001D0009053544F50914F4E54494D45924F4E4578
:1001E0005831935245544994444F95524553544F76
:1001F00052459652454D974E455854984F4E45524C
:1002000052994F4E9A494E5055549B524541449CE9
:10021000444154419D52455455524E9E49469F4734
:100220004F535542A0464F52A15748494C45A255FD
:100230004E54494CA3454E44A4544142A55448450C
:100240004EA6544FA753544550A8454C5345A95367
:100250005043AA4352AB49444C45AC535440AD4C77
:100260004440AE50474DAF52524F4DE028E12A2A4C
:10027000E22AE32BE42FE52DE62E584F522EE72EEF
:10028000414E442EE82E4F522EEA3DEB3E3DEC3CD3
:100290003DED3C3EEE3CEF3EB0414253B1494E5441
:1002A000B253474EB34E4F54B4434F53B554414EDF
:1002B000B653494EB7535152B8434259B9455850B5
:1002C000BA41544EBB4C4F47BC444259BD584259A9
:1002D000BE5049BF524E44C0474554C146524545A1
:1002E000C24C454EC35854414CC44D544F50C6495E
:1002F00045C74950C854494D455230C954494D45E8
:100300005231CA54494D455232C554494D45CB54DA
:1003100032434F4ECC54434F4ECD544D4F44CE52AA
:1003200043415032CF504F5254D050434F4ED141A1
:10033000534328D25553494E4728D2552E28D343EC
:10034000485228F052554EF14C495354F24E554CF8
:100350004CF34E4557F4434F4E54F550524F47F629
:1003600058464552F752414DF8524F4DF9465052BA
:100370004F47FF45585452412049474E4F5245443C
:1003800022412D535441434B22432D535441434B5F
:100390002275985A75891175885475C834758E10F0
:0E03A0009006FF745AF0E0B45A0974A5F0E01C
:1003AE00B4A5028003758E0C902001E493B4AA03C9
:1003BE0012209078FFE4F6D8FD753E4D853E81758E
:1003CE001380751411908000126DFBC39431F545A6
:1003DE00C2E2FFA312051812096AA31205189000B3
:1003EE005F126DFB900000B4A508E545C2E0640401
:1003FE006030BF02028003BF03071205FD80158027
:10040E0082AB83A982A3745AF0126DFBB45A05E431
:10041E00F0BBE0EDBB020040E690010A12056C1243
:10042E0005DB1205EF1213C1E545B4050312403981
:10043E00500F30E027908010126DFBB4551E02084D
:10044E008AE4FBF9780420B0FDD8FE12685F7802CA
:10045E0030B0F620B0FD30B0FD12096A906C091272
:10046E000632026AB8120482C28E85408D85418B97
:10047E00C28FD28E22C21712048B02130B12115A84
:10048E007C0150041210F8FC1204A4BC0013A385C6
:10049E00831385821422908010126DFBB4550ADCF2
:1004AE000122A3120506A380F0101DF5906BFF022A
:1004BE006C84126DFBFAA3126DFBF822CBC583CBB5
:1004CE00C9C582C922126DFBF540A3126DFBF54121
:1004DE0022D229121108120BF06017A320290E1236
:1004EE00052F120525126DFB202A07400512054522
:1004FE0080E4C22922900200D22980DA126DFBC05C
:10050E00E0A3126DFBF582D08322126DFBFBA312CA
:10051E006DFBF922120525C5827002158314C58262
:10052E0022C22A126DFBB5030CA3126DFBB125B5C9
:10053E000103B3B22AB3222582F58250020583222B
:10054E0012061CB1037406B14591CA90010812053A
:10055E006FB118900122B10A120B2C9001041205F2
:10056E006FEBF0A3E9F0A3221210ED900122B16F10
:10057E000E8E3F8060900104B10AB122126DFB60B5
:10058E0022A3B50711126DFBB5060BE5829402F896
:10059E00E5839400FA22E582C39409F58250DD15B5
:1005AE008380D912101DC3B199E89406F9EA94001C
:1005BE00FB900106B16FB12F4046D322126683A87D
:1005CE0004AA051266D9800BE513B402EF9002005F
:1005DE007401F0C215B14E90010AB118B1031205A3
:1005EE00FD9000FEE4F07511FE7509FEC21722A300
:1005FE00E4F0126DFB7009EBB583F4E9B582F022DD
:10060E0002689212115A50CD121150B449D33012C1
:10061E0002C2AA532220321206287D0D1207747DC3
:10062E000A020774D128E493C2E7B4220122D2341D
:10063E00FD120774A3800491CA7C0D1034E8126D6C
:10064E00FB6003B5040122B40DE6026C7A05A2909C
:10065E000007A8827D001207F6BD1B028003BD5B5A
:10066E002EB4440EE582B4070280E9B12512075478
:10067E0080E2B4430CE8B5820280D9A312076380EE
:10068E00D3B45B0280D0B41B047404800880C5B45C
:10069E001B03FD80C1FDB408028007B47F3DE8B5A1
:1006AE008211E582B407077D0712077480A6B12573
:1006BE00120754C082A3E8B58216120772D082E8E0
:1006CE00C39582C0E0120754D0E0D5E0F6188086BC
:1006DE00E0B125F0FD120774A380DAB40426E5829A
:1006EE00B4070CE8B5820FE582B4071102065D125D
:1006FE000754158280E8120772058280E6120754AD
:10070E00158280E3B40D088882F005A2020628B493
:0E071E0020005006120774020662B8500280D6
:10072C0088C08215820582120774E0CDF0E8B5828C
:10073C00F4D082E8C39582600AC0E0120754D0E07E
:10074C00D5E0F6A3080206627D1B1207747D5B12CE
:10075C0007747D440207747D1B1207747D5B1207BE
:10076C00747D430207747D20C0E0C083C0823035A5
:10077C00051207F180F8ED302C05122040803F3037
:10078C001C05124030803730270830190512403CC8
:10079C00802C301B2290012491D3C2979173EDD3FE
:1007AC007D0913308FFD92979173DDF6308FFD919B
:1007BC0073308FFDFD80073099FDC2998D99BD0D69
:1007CC0003751600BD0A0BE51560077D00F1741466
:1007DC0070F9BD08021516BD200040020516D08226
:1007EC00D083D0E022120832503230320512206011
:1007FC008011301E0512403380093098FDE599C2F6
:10080C0098C2E7B41302D235B41102C235B4030452
:10081C0030302822C228B41702D228D322D21D127B
:10082C00048B101D5922303203022068301E030243
:10083C004036A29822906D73120634C235120E28DF
:10084C001206281028EF302F2B020488E548A949FE
:10085C00B548F9C9954CE9954B2211584058D2141A
:10086C00C210A211922B9001268054121194850A69
:10087C0042850843D2179000F7D220026CA21205D1
:10088C00E1120DB7120BF060511211261211A012C9
:10089C000E34C22F853E81202F06850A42850843DF
:1008AC001207F1202F26B0185006900100F0D21834
:1008BC002014192010A43016132011109001207C44
:1008CC0002120CFED2111204C0020BEB1209F4122C
:1008DC00119450C0302F03026AD6026AC0B4D115ED
:1008EC0012113FB4245A120B48120FD712194C1282
:1008FC000B05020A25F50F121150B4CF0512114E3B
:10090C00C0E0120AEDE50FB4C317121142C2E5B4F0
:10091C005809121150758FFF0213C7758F000213FF
:10092C00C71210FBE50FB4C40990010A12056F023F
:10093C0005E3B4C50EA2AFC2AF8B48894992AF2272
:10094C00026C7AB4C8058B8C898A22B4C9058B8D4C
:10095C00898B22B4CA058BCD89CC22B4CE058BCB26
:10096C0089CA22120AFBB4CB0389C822B4C60389F4
:10097C00A822B4C70389B822B4CC03898822B4CD89
:10098C0003898922B4CF23D0E0B43003898022B408
:10099C003103899022B4320389A022B43306E9448E
:1009AC0003F5B022906B91026C84B4D093898722AA
:1009BC00BB09004003020ADE05A2C0E0E5D220E03C
:1009CC00FB900128E085F082858FF030F00225E065
:1009DC008582F0F5D3D0E089828B8375D202F075D5
:1009EC00D25075D2A005A222121142302D0FB42084
:1009FC0000500A122070121150540F805CB4C300C6
:100A0C0040030208E930E76FB4BC08120AFFBB00D0
:100A1C009FF722B4BD0B120AFF05A28B83126DE463
:100A2C0022B4AB004009B4B000500924F9801DB4C5
:100A3C00A4004003026C7A302F12B49000400DB425
:100A4C00A0028008B497028003B496E8121150906B
:100A5C00012CB480028091543F232582F582E493CB
:100A6C00C0E0A3E493D083F582E47312117A1212DE
:100A7C006012113950F52212112D405CC21512046E
:100A8C00CA7FEA120EF4121142B42214AF3F1211B3
:0E0A9C005012115A609EF0B4222B740DF0021D
:100AAA001150C083C08212112D408BD000D002AFEA
:100ABA003F126866B40D0122DF08740D126DF3024D
:100ACA00108A1267C480EADF0851A612108A02113E
:100ADA0065A380BC906B7B026C84120AEA021263E3
:100AEA0012117AC002C0007FEA1211BFD001D003EE
:100AFA0022BB00E022121150120EED51ED121935EF
:100B0A00EEBF00D02212110051FB09E960C6900124
:100B1A0004853FF0120B3A90010A12688D853F82D4
:100B2A001583C3E99582F9EB9583FB492275F00693
:100B3A0012050AE9A42582F9E5F03583FB22710F33
:100B4A00C003C0017F2C120EF41210F8E9B53F0061
:100B5A00508219D0E029F9D00350010B020EF2514C
:100B6A00EAC003C0011212637FA61211BF1211421A
:100B7A00B4A7081211501211C280031218C174EFDF
:100B8A00120D94120DA07B00A900121263121263B7
:100B9A0012110FA801120D03D008D00A7C01120D00
:100BAA00031211260208A01211C212113950F8229A
:100BBA0012117A12126012113950F522120C19F917
:100BCA00121142B4A503121150B9000D7FA81211D7
:100BDA006760E8121150B4A8F31211B35003020966
:100BEA00F4120C24800B126DFB1420E73622120C2F
:100BFA004D1211261025093015031205E102089E2F
:100C0A001014055322BD8004A22B92110208A012CF
:100C1A0011C2121645600274FF22121108126DFBEE
:100C2A00FFDF06906BEB026C8420E7F7A3126DFBE3
:100C3A00B5020AA31F126DFBB50002A322EF12052B
:100C4A004580DA1211ADC013C014C083C0821211DC
:100C5A0042B42C161211501211ADB80008751302C5
:100C6A007514008005AC00120496D082D083AA8342
:100C7A00A8829124121194D001D003229119F480F0
:100C8A000291197C03FD800E1211AD88150208E647
:100C9A00D2257C027D55120D1E126DEAF5830812CB
:100CAA006DEAF58208126DEA6010B4040D08126D3F
:100CBA00EAF51308126DEAF51408126DFBB4010384
:100CCA000208E6ED60068811F4700122020BFB911E
:100CDA004DE9B51406EBB513028011C00AC0088BA2
:100CEA000A89087C04120CFED008D00A7C02120C75
:100CFA00FE020BAB74FD120D94E50805A275830084
:100D0A00126DF518E50A126DF318EC126DF32274E0
:100D1A0003120D94A81105A2758300126DECB50497
:100D2A000208226076B401E7120D9280E77C01B1D5
:100D3A001E880F790B126DEAF70908B90FF7120F1F
:100D4A008A5004AA0BA80CEAB50B50E8B50C4C1251
:100D5A00126D740E250FF87A0005A28A83126DECC3
:100D6A0008C0E012126DC00012146A1218A2AB0B6E
:100D7A00A90C1212637A00D00012126D126004D00C
:100D8A00E06001B372D5401974112511B4610040B5
:100D9A000AC51114F82212119450FA900389026CB0
:100DAA0084850D0A850E080208A0120DC0121108CA
:100DBA001211261211A0C50AC512C50AC508C51006
:100DCA00C50822B1C0121139401C1211C2121142B7
:100DDA00B42C028003121194B1C012117A1212605B
:100DEA0012113950DE22B49C0512115080DCB40174
:100DFA0008B1C0906BB7026C84121165121194404D
:100E0A00F080C2121142B42304D21B8005B440D52B
:0E0E1A00D21902113FD236D237D10D120E2F4F
:100E28005323F553263F2212115A4008020628126E
:100E3800113940F812111650F6B4A4091211009590
:100E48001640EC8006B4A90B12110060E21207727A
:100E58001480F8B4D31812113FB4240812128A125D
:100E680010FB80061210F8120EF2AD018008B4AA29
:100E78000A1211507D0D12077480B4B4D25E12119B
:100E88003FB446187517F012113F121150540F60F5
:100E980007B40300500274034217802FB43008755A
:100EA80017001211508024B42321120ED98F17B4C1
:100EB8002E1412113F120ED9EF251724F7500302F2
:100EC8006C7AEFC44217E517C4F517120EF2020E3A
:100ED800377F00B4230E0F12113F80F712115C50B8
:100EE80003B4A843227FE01211BF7F2912114EB527
:100EF80007CD221210F812114EB48306120F1302F6
:100F08000BABB49FBA120F13020CF6B9000B1211F7
:100F1800AD12116591240211947F2C121167B42C23
:100F28009E1912115080E412112D40061206450236
:100F38000E371211C27448B516005002D13430373A
:100F4800161215E940111217CE70091210FB126023
:100F580016020E371217E612600E7401020E5312B3
:100F6800113F126679400CB45F0122B4410040047D
:100F7800B45B00B32230D541906BAC026C84D2D5FF
:100F88008002C2D5121142F173500420D5EA22FF23
:100F9800E4FDFEF1674007CF2DCF7D1A80F4C2151E
:100FA800B4E033430680120583C002C00050C62057
:100FB800D52C790A7B00120FF9121103BB00B9D0A6
:100FC80082D083126DFB149940AE1205227137C985
:100FD800C8C9CBCACB2220D59F120583C3221211C0
:100FE80003BB0094D000D002120FF9121139508EB1
:100FF8002209E96083FC900108120B37AF83AE82A7
:1010080090010612688D90010812056F88828A8304
:10101800ECF0120522EFF0A3EEF0221211161211D5
:10102800395008120E347D3F120774D22212065B23
:10103800C222750F00750E0712112D4010120FD71E
:10104800AB0FA90E120AB912113950DA22126C42EA
:10105800126D5C701D126C4912117A121260126CBA
:10106800421211394015126DFBB42C06A3126C49BB
:1010780080C69000FC120632026C39126DFBB40D6A
:101088000122900373120632020E341210ED8B4BBC
:10109800894C900126D21002101D120F8A4010129E
:1010A800126D12160FA801AA0388828A8380031280
:1010B80011ADBA000AE820E70628904100F582122F
:1010C8000A7553D0E7223031323334353637383960
:1010D8004142434445461210F81213EA8B408941B5
:1010E8007F2C120EF41211C27F2C1211BF02193577
:1010F8001211C212160FE922121150120EED80F3CE
:1011080085138385148222850A8385088222121119
:1011180042B4221A310FA37C22120649A3C3858345
:101128000A85820822121142B4246B020B0F0211A5
:101138009E121142B42CF7121150D2D305A28A8301
:10114800126DECC2D3223142D2D308B800010AC2D0
:10115800D3223142B40D02E422B43A3A227F0D314F
:101168005A50F9B5070122315080F43150315A7084
:10117800FA22120F8A8031120DA07C03120CFE0293
:1011880008A0B43A0280C1B4A87231753142B40DD6
:0E119800F1313FB40102D322C5082403C5087B
:1011A60010D70122050A221211B3405222310F1222
:1011B600601231268A83888222120EF47AD8C002FF
:1011C600C224E581240C5003026C81E50994385051
:1011D60003021604202416120F8A500E1212805093
:1011E6000C3142B4E00774D9806112126D3142B4F9
:1011F600E000500EB4B000503CD0022024BAC30226
:101206006C7C541F202405B40548740924D9FA902F
:10121600000093FCD0E0FD93B50404B40C9AD350BF
:1012260097C005C002315031C4D0E0900060242739
:10123600120A65808D3150B4CF05314EFA74CF2035
:1012460024BC243940E5B4F70050E0C0E0120EEDAE
:1012560080D7B403A931500211C8120FD712164510
:101266000218FA7A0178131215F5D2240218FA1127
:10127600F880EA11F8120FD780ED3142B4D113315C
:101286003FB42406120B48021803121949315002C2
:101296000EF2310F126D5CB4FF02D3227006C3D278
:1012A60024021126540B60F3906B9C30E003906B84
:1012B6005730E103906BBF026C84120E0D121814A6
:1012C60031B3E4FBF94014126C49314EB4E508120F
:1012D600164531AD12194CAB0FA90E1204E160256B
:1012E60051A7A31213BB1215F2401A1207F11215D9
:1012F600F5310F12131C51A712130EA3126DFBD555
:10130600E0DE121645026AC0900007120647310F4A
:101316000206281204CA7B007907A351A71204C04B
:10132600126010310FA3B90D004028A3126DFBFE09
:1013360020E72AB420005003B40D22B4220B121366
:10134600AB1213AEB422FA80DDB43A0C1213A9EE36
:101356001213AB1213A980CE1213B280C951A7A2E1
:101366002D92D590017E30D503122078E493A3B454
:10137600FF0610D5EE026AC0B506F1B4B000500300
:101386001213A9E49320E70860061213ABA380F3B7
:10139600310FEE649670051213AE80FB508812135F
:1013A600A980837420026938A3126DFBB40DF6027E
:1013B600692090010A1204C002194C9015091218EE
:1013C600AA12189F90150312160A900128E9F090A8
:1013D60014FD12160AE9F404F54A7B017913021288
:1013E6006312160AE9F4240FF9EBF43400FB221118
:1013F600DE71EAC292C28E8B8D898BC28FD28E121B
:10140600693D308FFD1217F5D292120476308FFDAA
:1014160070E122516931C2740C12194912158512F4
:10142600187E12160F71EA90012402056F71B81228
:101436000503A882AA8312194C1260020212AA128C
:101446006A93AA07EE02194BA2AFC2AFC047AA48D9
:10145600E54992AF12194BD0E012194974C8121916
:101466004912187E1260000212AA7E0057226628D0
:101476007F01375716167F00149690427F014096DB
:1014860028758000646265108001998820148000A8
:101496005135991980014531333381000000001020
:1014A600FF8100000000208000713713197F00764D
:1014B6006437948000072275178000523593288080
:1014C6000071918586FF8100515802237700449070
:1014D60005167901082105257B00197355277D011D
:1014E600701284197E003333338380016766661673
:1014F600810000000010FF7B00006127167B0000C2
:1015060000005088000092051185004241875981EC
:0E1516000018281827810026594131000000D6
:1015240000000085000050536512155D916A121980
:101534001012158BE546540162451218A212155D6E
:101544001215F24005121910913F1217CE9014D2C1
:101554001215691215BA0215E21219109014A71285
:1015640018AA02187E12189F1215851218C612188E
:10157400AA1218CD1215851218AA916AE493B4FF21
:10158400F01260060212AA1218F312187E1217CE75
:10159400F54512189F12160FC00389461217A5911C
:1015A4003F1218D4B185D003221218A2B1321218F6
:1015B400D8B12D02187E1216497B010217BA1217F0
:1015C400CEF545121649247F922A500312167C90B8
:1015D4001470B169302A071217E6B15D916AE545C6
:1015E400601D0217E61218A21218141218D802600D
:1015F4000474FA2509B432004006F509F97B012286
:10160400900381026C841218AAB185E4FBF9A8093D
:1016140005A2758301126DECC39481FC18126DEA66
:101624007068401D0CE89405F808126DEAC4126055
:10163400144057DC02800A126DEA126014404BDC3D
:10164400E874068001E4A8097A0105A28A8305A248
:101654002840ADF509126DEA221218C1B18BBB0006
:10166400291218F3D1451218C61218C1E546701193
:10167400E54560E490011EF01218C11218D8021852
:101684007E15461218CDB18580E2020ADE1217CE0D
:1016940070F81218F31218C67819126DEA602B2428
:1016A40080500503547F8007F40403547FF404241A
:1016B40080126DF31218D41218CD12187E1218CDA0
:1016C400916AB16012173E30D5EA0218CD1217CED6
:1016D40070B8F54608126DEA60B0B48100922A40F1
:1016E40002D17C1218A21218C1B1F2501FD14924A0
:1016F40085500F1218A774012546408EF546B18512
:1017040080E190150F1218AA740B80EC1218F312D2
:1017140018C1913F1218D41218C1916A12187E9000
:1017240014ADB169A31218AAB185E54612194991FD
:101734003FB1BA302A01220217CE1218CD1218D89E
:101744001218A21218C60260041218A71218D8D1CF
:101754005D90011F126DFB60DD1218D41218CDD1FB
:10176400496002D1D1B1851218A71218D8D15D757C
:1017740046001218C11218A21218C61218D4B18544
:101784000546E54612194912187E1218A21218CD00
:10179400916AF13E30D5E4D1451218CDB1850215D8
:1017A40085D14994815008D1459015210218AA94F5
:1017B400075016F404FB1818126DEA54F0126DF376
:1017C400DB0122E4126DF3DBEE221217E670221223
:1017D4006DF322D14560D218126DEAFF1218C1EFE1
:1017E400600FD14918600A126DEA6401126DF36446
:1017F4000122D10F1204CAE49302194912160F05EB
:10180400A28B83126DDB0219491215F272D540992D
:101814009015270218AA1215F2B380F21215F2A23B
:10182400D580F61215F2B2D580F51215F280DF12CA
:1018340015F272D580E312160FBB0004E7021949B2
:10184400BB09004003020ADE05A2E5D220E0FB75D5
:10185400D20289828B83E075D20005A202194990D5
:10186400010C120518E9C313F874061329C83BFACE
:10187400158212189912194C11141260080212AA36
:101884001211ADD213900102800B1211ADD212438A
:0E189400A884900120EAF0A3E8F0221218A226
:1018A200121649802A9015151215F505A28B83058B
:1018B200A27B06E493126DE2A319DBF7D2242290F5
:1018C20014F680E47B01791902126378197A010215
:1018D200126D781F80F71216497406FA28F9126DF4
:1018E200EAFB126DD9126DF3EB126DE21918DAEE02
:1018F200221216497B01791F7C0605A28A83126D8A
:10190200EC05A28B83126DE412685BDCED2290156C
:101912001B8095121935EB5FFAE95E802C1219359E
:10192200EB4FFAE94E80221114121935EB6FFAE9E6
:101932006E801612160FAF03AE0102160F90010051
:10194200126DFB101801E47A00F8D224026018E547
:10195200A880F4E5B880F0AA8CA88A80EDAA8DA8A8
:101962008B80E7AACDA8CC80E1E5C880DAE5888043
:10197200D6E58980D2AACBA8CA80CFBA3004E58046
:1019820080C5BA3104E59080BEBA3204E5A080B7C2
:0E199200BA3304E5B080B00209B0E58780A941
:10600000012A011A01F121262164614C618A814D26
:10601000A1F5A199A1D1C146617B05A2758301A813
:106020000918126DECB2E0126DF3126323EF6012E7
:10603000BE00171263137F06126DEA126DE2181983
:10604000DFF6E5092406F509E4229E8F308C2F50F7
:10605000098E308B2FF404C8C9C8FFC223BD0002CB
:10606000D22312633CBF0B0040027F0A752A001244
:1060700062707F04792E749EC39CD4CC7001FCB4F2
:10608000500030231EB3126098500A052A7F011277
:10609000627012622102620F126DEA37D4F718198A
:1060A000DFF622126DEAFEE43499972ED4F7181920
:1060B000DFF14011B278792E7F04749A972400D4CE
:1060C000F719B3DFF5782B7F00E670090F0F08B8DA
:1060D0002FF702625FB4100050010FE530C39F60DC
:1060E0000D400BF5301262AA752A0002620F02629F
:1060F00058126323E509240CF509EEC2D59F600A06
:106100004003EB8001EC6001B322BD00F57F041871
:106110001818191919126DEAFE126DD99E70E60849
:1061200009DFF2D2D522126321BE000302625F8D25
:106130002FEF60F82E20E70610D7080262585003B0
:106140000262479481FE12622D7B04AC018C011225
:106150006DD9FA1262E0EAC41262E01CDBEF8E3005
:106160008D2F80691263238D2FBF0007126247E4D1
:10617000D2E322EE60B69F20E70550050262585038
:10618000BF2481F53012633C7A34AB00752A007D60
:10619000FFD38B00792E7F045019126DEAFEE43490
:1061A000999E27D4F71819DFF10D40E6E79401F71F
:1061B000B380DF119877008A00A6050A7F0112627A
:1061C000A8BA3ECBD53003026258752A007834E66F
:1061D000FE600412622118087408F928F8B6050058
:1061E0004014D3E41836D4D630E40AD9F518760131
:1061F000126221800619E9C3C898F8792BE6C40811
:10620000D64206F70809B92FF4EE70037530001274
:10621000631389097830E6126DE21819B82AF7E499
:10622000220530E53070F9D0E0D0E0801AC0017965
:1062300032126DEA540FF7126DEAC4540F19F718B1
:1062400019B92AEDD00122782E7499F618B82AFBD4
:106250007530FF510FD2E12212625FE4D2E02212C8
:106260006267510FD2E222E4783DF618B829FB228A
:106270007C00C3EF60229402501FC000C001792E41
:10628000782DECD7C4FCE7D6C4F71819B92AF7E77C
:10629000C4540FF7D001D00022FFE4C52AC52BC596
:1062A0002CC52DC52EFC80CB7C00C3EF6022940250
:1062B000501FC000C001782A792BE6C4F6E7C4D687
:1062C000F70809B82EF7ECC4D654F0FCD001D00082
:1062D00022FFE4CCC52EC52DC52CC52BC52A80CBED
:1062E000540FFF783C7932E4F5331826D430E403B8
:1062F000180608D68FF0E7A475F00A84C5F026D4F6
:1063000030E40205F008D618E5F019B92ADC253387
:10631000D4F62205A275830105A2A809740628F9FE
:106320002251677113126DEAFF126DD9FE1819120E
:106330006DEAFC126DD9FB6CFD181922C000782E95
:10634000126DD9F61918B82AF7D00022126430C09D
:1063500083C082126DFB126679401112636F400C8C
:10636000B44803D38001C3D082D08322A380E4C287
:0E637000E5B447005004B44100B3227B00792D
:10637E00581265F5740D126DE29000585167126453
:10638E0030126438927878347E7FD2D51266775088
:10639E0008540F126409A380F3B42E0C205168D256
:1063AE0051B834F2D25280EE20D55CB4650280032F
:1063BE00B4453712642F12643892501266775047E4
:1063CE00540FFDA3126677500D540FCD75F00AA42D
:1063DE002DFD50EF7DFFED305009C39EF4044009B2
:1063EE007401222E5003740222CE8E30B834025124
:1063FE0067E509C3940CF5090261CDC2D5700BB8DF
:10640E003408305204DE0274FF22205302C252209E
:10641E0052F32051010E2053F0B83D02D253F6082C
:10642E0022A3126DFBB4201680F7B4E302800EB4E3
:10643E002B028009B4E5028003B42D02D3A322718E
:10644E00231142EFFE512D782BE517FB6057B4F068
:10645E000040030264EBEE70027E80EBC4540FFA30
:10646E0012655FCAC39AFF50077D3F12659680354D
:10647E00BA00091F1265831265908008126583EABF
:10648E00FF126542EB540FFA60B412658C12656808
:10649E00B50204EA02657950FACAC39ACA1265793E
:1064AE00EAFF026542EE70061265940265907BF07B
:1064BE0074772E402894F7402412658512655FB4D8
:1064CE0008028070126542126555606712658C7FF6
:1064DE0001126542705D126555605880F212658535
:1064EE007F0112654212658CEB540F6007FF1F127D
:1064FE006542800291DD1265947D45126596EE60CF
:10650E000414B48006126594E4800E40077D2B12AD
:10651E0065968005126588F404C2E7F87A0079580A
:10652E007B001265F57858126DEAFD12659608E843
:10653E00B501F422EF600FE64430081FFD12659698
:10654E00E4B833F0745522A900E7700409B933F9A1
:10655E0022EEC394805001E4FF22C374809E50014A
:10656E00E422EF60FC1265941F80F7FFEF60F212D9
:10657E0065901F80F7B170EC600C7D2D800A7D2E2A
:10658E0080067D3080027D20020774714C922312AA
:10659E006677B3402A7B0079008016A389008B02B0
:1065AE00126677400C302317716F4003A3801024BE
:1065BE000975F00A30230375F0101265D450DCE42F
:1065CE0092E12275F00AC0E0C0F0E9A4F9EBABF05D
:1065DE00D0F0A4A2D292D52BFBD0E072D5400754B6
:1065EE000F29F9E43BFB22E4902710126617900363
:1065FE00E812661790006412661790000A1266176A
:10660E009000011266176020227EFF0ECAB583002D
:10661E00CA4012C89582C8CA9583CA50EEC8258250
:10662E00C8CA3583CA4E60E074302E05A28B831221
:10663E006DE409B900010B22B194A2369223EB123C
:10664E00666EEB12666FC223E912666EE912666F12
:10665E007D488009C2232490D43440D4FD0265962F
:10666E00C4540F70EF3023EC229130B43A00500432
:10667E00B43000B322908010126DFBB4550BA3AC56
:10668E0082AD83120506A380EFEDB5130CECB514A5
:10669E000812052522D183800B0204BAE513B40239
:1066AE00F4120503AC82AD83AB0FA90E1204E17098
:1066BE0031E50DB4040122126880AA05A804126700
:1066CE0044E513B40205740102686DC00EC00F8854
:1066DE000E8A0F7401126A3F74FF126A3FD00FD0F8
:0E66EE000E22FF126C49E50D4009B40401E4D0
:1066FC009F603B4022FFE50DB4040122EF1268803D
:10670C00126C42126875120FD7A904AB050EBE00AD
:10671C00010F1268498017F404120545126875A917
:10672C0082AB83AA0FA80E6003126750D1CFAA0FB9
:10673C00A80EE50DB4040122E47904FBAE0DFFE5CF
:10674C0013B40211E513B402181268661267C4126E
:10675C00693D70F522880E8A0F1269D1A80EAA0F16
:10676C0022C00EC00F7480BF0008B5060280034023
:10677C0001EECEC39EC0E0E4CF9FC0E089828B8344
:10678C0005A2900063A982AB8305A2AC06E493A397
:10679C0005A2F0A305A2DCF5C082C083880E8A0F87
:1067AC001269D1AA0FA80ED003D001D007D006EEE3
:1067BC004F70B2D00FD00E2208B800010A09B900F0
:1067CC00010B22F1C4C00EC00FC000C002880E8A9B
:1067DC000F74FF126A3FD002D000E8547F04BF0050
:1067EC0008B5060280034001EECEC39EC0E0E4CFA4
:1067FC009FC0E0E8C39EC0E0F50EEA9FC0E0F50F35
:10680C00E9C39EC0E0F582EB9FC0E0F58305A29042
:10681C000063A982AB8305A2AC06E493A305A2F0A6
:10682C00A305A2DCF51269D1D003D001D002D000AF
:10683C00D007D006EE4F70A2D00FD00E22E513B4C5
:10684C00028112686612685B12693D70F0002218B2
:10685C00B8FF011A19B9FFF51B2205A28B83126D23
:10686C00DB05A28A83126DF522ECC39582FEED95B1
:10687C0083FF4E222CF9E43DFBE513B4020E90018C
:10688C000412052F40ED906B69026C84BBFCF58003
:10689C00F3126AA51211B3126C4992D5900005122D
:1068AC001899A8087907C22490017E8805E493FF03
:1068BC00126DEAFBB461004007B47B005002C2E5E4
:1068CC00FA126DF3A3E493B502030880E320E731D9
:1068DC00602FA3E49320E70370F8A3A805B4FFCBC3
:1068EC00BA20030880C0302D0A202407D22412209D
:1068FC007880B812691DB422AD12691DB422FA80D9
:10690C00A5EF126938B4969EEB12692012691D80AE
:10691C00FB126DEAB40D14D000D000126DE20974B4
:10692C0001126DE2E99404F50D790408126DE20987
:10693C00221EBEFF011FEF4E22750F80750E00B494
:10694C00300274FF126A3FE5CB126A3FE5CA126A45
:10695C003F90010AE0126A3F90010BE0126A3F027D
:10696C0069CE880E8A0F0269D11211B34013AC00A4
:10697C00BC0015750F80750E1074FF126A3F02690A
:10698C00CE12115A70B37CFEC004D21D1204A41294
:10699C006C49D0E0BC000280011C9C1219491260A9
:1069AC000E126A93120628EB20E77F7455126A3F89
:1069BC001269D174FF126A3FA90EAB0F1266461210
:1069CC000628020488E50E547FF4042480BF0008D6
:1069DC008E00B500004001EE605005A28B838982C9
:1069EC0005A2C0E0750009126A5BD000C3EE9500E9
:1069FC00FEEF9400FF850E82850F8305A28B8389A1
:106A0C008205A2E493A3F50205A2E0A305A2B502B8
:106A1C0019D500EF85820E85830F05A2A982AB8361
:106A2C0005A2EE4F709F53D0E72253D0E7906BD066
:106A3C00026C847802C0E0126A5B850E82850F833B
:106A4C00E493D000B500E3A385830F85820E22C0AA
:106A5C00A8C2AFCEC0E0EFC0E0E9C0E0EBC0E0EE12
:0E6A6C00A900850E82850F8375A22012FFF00F
:106A7A0075A200FED0E0FBD0E0F9D0E0FFD0E0CE76
:106A8A00D0A82275D018316E221204DFA3AB13A945
:106A9A0014C3E58299FEE5839BFF22750A007508F7
:106AAA00072251937A0278001267551205E3C2173A
:106ABA00751302751400120E28C22DE49020029359
:106ACA00B45A03122048900106120632D22F853E8C
:106ADA0081121316C21890005E126DFB64347003A3
:106AEA0002088A7D3E12077412065B119D20D54169
:106AFA00900007E0B42E2AA3E0B40D25AB0FA90E2F
:106B0A001204E1302A1B12131C7D3E1207749000F6
:106B1A0007E0B40D0512066080D1FD120774A38048
:106B2A00F01266AA12054E2015AAD2151205E380A4
:106B3A00A351A512115A6094900118B4F000400AAA
:106B4A00121150540F120A6580820208A09E415207
:106B5A004954482E20554E444552464C4F57224DD3
:106B6A00454D4F525920414C4C4F434154494F4E89
:106B7A0022A842414420415247554D454E5422498C
:106B8A002D535441434B224241442053594E5441C0
:106B9A0058228A444956494445204259205A455266
:106BAA004F2241525241592053495A45224E4F20B1
:106BBA0044415441229441524954482E204F56454B
:106BCA0052464C4F572250524F4752414D4D494E13
:106BDA00472243414E275420434F4E54494E554570
:106BEA0022494E56414C4944204C494E45204E5567
:106BFA004D4245522250524F4D204D4F4445222A74
:106C0A004D43532D353128746D2920424153494350
:106C1A002056312E342E62657461342F5244322A42
:106C2A00224552524F523A2022906BDC30174B8544
:106C3A00420A85430802089B850F83850E822285B6
:106C4A00830F85820E22202F27C2964387012016A2
:106C5A000B1021083010F412085840EFD29622A3E4
:106C6A00202F233013209001011205F3A30208D22A
:106C7A00A22F906B918004906B89C3853E81120E7E
:106C8A0028E49310E7D9914940031205EF1206252B
:106C9A00906C2B1206349142120634302F05C22012
:106CAA00026AC090010C120634121108E4914912CA
:106CBA000545126CF740086006126DFBB401EE91AF
:106CCA0042126CF7E9240AF545A31213BB12600EAF
:106CDA002020CB120625914212131C12130E7D2D71
:106CEA00120774D545F87D5812077480B1AB0AA90A
:106CFA0008020B2C854A8CC54704B4C808E4054928
:106D0A00B549020548C547D0D032126D37C2A9C26B
:106D1A002E500D5389F0438901D22E43A882D28C7A
:106D2A0022126D37921E22126D37921C2212114EB8
:106D3A009431B32220D4FC20D3F910E706900050F6
:106D4A00020A6520E0066007905FFE7302638A020A
:106D5A00077412600A50F5126012700CC083C08268
:106D6A00126018D082D083E422D7D2C9D454C5CEB7
:106D7A0020C2D920CACFC8CEA04BC1D4C1D553CBCB
:106D8A00D92C2049CED4C5CCA0C3CFD2D02E203105
:106D9A00B938350D0ACD6F64E9E6696564A0E66F16
:106DAA00722052C43220E27920F7E56B20A84329E9
:106DBA00B2B030B42D36202020A0A0E87474F03A86
:106DCA002FAFF7F7772EE56674EFEEAE73EB220579
:106DDA00A28982B1FB05A22205A28982F005A2221C
:0E6DEA0005A28882B1FB05A22205A28882F0D4
:0D6DF80005A222E58330E703E49322E022A8
:00000001FF
